:020000040000FA
:0A0000000000000029EF00F03CD0E2
:0800180091D09EA8FED7AD6E49
:1000200012000B6A0A6EFF0E0A260B2200D0D8A01F
:100030001200030E096EE60E02D8F5D7096AFE0F0C
:10004000086EE86A095AD8A012000000080600D01D
:10005000F8D7006A4F0EAF6EB06A240EAC6E900EE9
:10006000AB6E00010F0EC16E070EB46EC69AC00EC5
:10007000926EE00E936EC00E946E956AE80E966EC8
:1000800070D09EAA1BD0060EAB1412E1E2CF2EF068
:10009000E1CF2DF02F2A10EE36F02F50E126000E82
:1000A000E222AECFE7FF2EC0E2FF2DC0E1FF11003C
:1000B000AE50AE50AB98AB8811000BD0F2A409D073
:1000C000F294104A112AD6CF0EF0D7CF0FF08176D6
:1000D000110011002F50305C14E0302AEACF09F0F3
:1000E000E9CF08F000EE36F03050E926000EEA22A3
:1000F000EF502C6E09C0EAFF08C0E9FFD88012005B
:1001000004D0E8682C6ED8A0120012002F6A306A62
:100110009D8A9F8AF28EF28C12009D9A00EE36F034
:10012000010EF46EF36AF306000EF45AEE6AF45010
:10013000F310F9E12F6A306A9D8A1200F29EE0CF37
:1001400063F4D8CF64F4E8CF65F4F28E0001A19295
:10015000F29E63C4E0FF64C4D8FF65C4E8FFF28E7A
:10016000100093968A860A0E5CDF93968A96929286
:100170008992929A899A9296899695988C98949851
:100180008B9895948C9495908C9094948B94949057
:100190008B9096928D929290899092988998929451
:1001A000899496908D9094928B9295928C9295963C
:1001B0008C9696948D9494968B96949A8B9A93920F
:1001C0008A9207EC07F0BFEC07F0356802EE41F0C9
:1001D000200EEE68E82EFDD7256A0401628196DFC5
:1001E00000019BDFCD6AF294F28A870ED56EB16A68
:1001F000A192A082B36AB26AD08EA292B10EB16E01
:100200004A0E2B6E400E2A6E0201376BBC0E05DFC4
:10021000420E03DF400E01DF0001D6CF0EF0D7CF34
:100220000FF058DF2CC016F0CD0E165C07E3FE0E63
:10023000165C01E301D0186A2DEF04F016AE38D039
:10024000186A8C0E165C05E116C018F019681A6859
:100250002DD09C0E165C05E116C018F01B681C68BA
:1002600025D0AC0E165C05E116C018F01D681E689E
:100270001DD0BC0E165C05E116C018F01F68206882
:1002800015D0CC0E165C04E116C018F021680ED013
:10029000DC0E165C04E116C018F0226807D0EC0EE4
:1002A000165C04E116C018F02368246828EF04F0F7
:1002B000185204E12DEF04F028EF04F08C0E185CC6
:1002C000D8A490D0192803E116C019F089D016C01F
:1002D0001AF0340E195C37E35F0E195C34E2020148
:1002E0003753000127E0D50E8016020144694369A7
:1002F0004269416903EE62F0D8902A34E926000E83
:10030000EA22EECF06F0EFCF07F006500E24026E81
:1003100007500F20036E000E1020046E000E1120F7
:10032000056E05C048F204C047F203C046F202C0A1
:1003300045F2618102013A6B04016231000102E37E
:100340008D948D904CD0790E195C09E102014C69B5
:100350004B694A6949698D946181000140D0780EEA
:10036000195C09E1020150694F694E694D698D9030
:100370006181000134D07A0E195C09E102015469EF
:100380005369526951698B926181000128D07B0EBB
:10039000195C09E1020158695769566955698B96DC
:1003A000618100011CD07C0E195C09E102015C69CD
:1003B0005B695A6959698C926181000110D07D0E88
:1003C000195C09E1020160695F695E695D698B9A88
:1003D0006181000104D07E0E195C01E18C961968E0
:1003E00028EF04F09C0E185CD8A404EF04F01B283E
:1003F00004E116C01BF003EF04F016C01CF01C5201
:10040000D8A487D0340E1B5C37E35F0E1B5C34E24C
:1004100002013753000127E0D50E8016020144691E
:1004200043694269416903EE62F0D8902A34E926B3
:10043000000EEA22EECF06F0EFCF07F006500E24B2
:10044000026E07500F20036E000E1020046E000E87
:100450001120056E05C048F204C047F203C046F201
:1004600002C045F2618102013A6B04016231000170
:1004700002E38D948D904CD0790E1B5C09E1020152
:100480004C694B694A6949698D946181000140D08A
:10049000780E1B5C09E1020150694F694E694D6994
:1004A0008D906181000134D07A0E1B5C09E102015C
:1004B00054695369526951698B926181000128D056
:1004C0007B0E1B5C09E10201586957695669556941
:1004D0008B96618100011CD07C0E1B5C09E102013E
:1004E0005C695B695A6959698C926181000110D01D
:1004F0007D0E1B5C09E18B9A020160695F695E6990
:100500005D696181000104D07E0E1B5C01E18C9667
:100510007AD1340E1B5CD8A045D05F0E1B5CD8B0DE
:1005200041D001EEB7F01B50EB50026E0201375D77
:10053000000129E001EE37F01B50EB500201376F4C
:10054000C00E80163751801202EE62F0D8902B3424
:10055000E926000EEA22EECF06F0EFCF07F00650B4
:100560000E24026E07500F20036E000E1020046E42
:10057000000E1120056E05C044F204C043F203C012
:1005800042F202C041F21BC03AF2020148694769D7
:1005900046694569618104016231000102E38D848D
:1005A0008D8030D1790E1B5C2FE18D847F0E1C5C19
:1005B00022E203EE62F0D8901C34E926000EEA2213
:1005C000EECF06F0EFCF07F006500E24026E075074
:1005D0000F20036E000E1020046E000E1120056E19
:1005E00005C04CF204C04BF203C04AF202C049F20B
:1005F0001CC03BF205D002014C694B694A6949694C
:10060000020161810001FED0780E1B5C2FE18D801C
:100610007F0E1C5C22E203EE62F0D8901C34E926C7
:10062000000EEA22EECF06F0EFCF07F006500E24C0
:10063000026E07500F20036E000E1020046E000E95
:100640001120056E05C050F204C04FF203C04EF2F7
:1006500002C04DF21CC03CF205D0020150694F6946
:100660004E694D69020161810001CCD07A0E1B5C9C
:100670002FE18B827F0E1C5C22E203EE62F0D890A9
:100680001C34E926000EEA22EECF06F0EFCF07F089
:1006900006500E24026E07500F20036E000E10202D
:1006A000046E000E1120056E05C054F204C053F212
:1006B00003C052F202C051F21CC03DF205D002014B
:1006C00054695369526951690201618100019AD0EC
:1006D0007B0E1B5C2FE18B867F0E1C5C22E203EEFF
:1006E00062F0D8901C34E926000EEA22EECF06F024
:1006F000EFCF07F006500E24026E07500F20036E56
:10070000000E1020046E000E1120056E05C058F278
:1007100004C057F203C056F202C055F21CC03EF2AC
:1007200005D002015869576956695569020161810E
:10073000000168D07C0E1B5C2FE18C827F0E1C5C5C
:1007400022E203EE62F0D8901C34E926000EEA2281
:10075000EECF06F0EFCF07F006500E24026E0750E2
:100760000F20036E000E1020046E000E1120056E87
:1007700005C05CF204C05BF203C05AF202C059F239
:100780001CC03FF205D002015C695B695A69596976
:1007900002016181000136D07D0E1B5C2FE18B8A46
:1007A0007F0E1C5C22E203EE62F0D8901C34E92636
:1007B000000EEA22EECF06F0EFCF07F006500E242F
:1007C000026E07500F20036E000E1020046E000E04
:1007D0001120056E05C060F204C05FF203C05EF236
:1007E00002C05DF21CC040F205D0020160695F6981
:1007F0005E695D6902016181000104D07E0E1B5CAF
:1008000001E18C861B6824D0AC0E185C0AE11D281F
:1008100003E116C01DF003D016C01EF07AD91DD01A
:1008200017D0BC0E185C09E11F2803E116C01FF0A9
:1008300003D016C020F092D90BD0CC0E185C08E182
:10084000212806E116380F0B216E215201E063D9F1
:1008500002016131000101E31FD9080E355CD8B0F7
:100860000DD131500E5C32500F5833501058345067
:100870001158D8A002D1348E35520DE1C00E801629
:10088000D890020137333751801244694369426975
:1008900041690001F1D0010E355C0BE1C00E8016FC
:1008A00002013A6B376B486947694669456900013F
:1008B000E3D0020E355C23E1847403EE62F0D8903D
:1008C00002013B35E926000EEA22EECF06F0EFCF1B
:1008D00007F006500E24026E07500F20036E000E24
:1008E0001020046E000E1120056E05C04CF204C0ED
:1008F0004BF203C04AF202C049F20001BDD0030E20
:10090000355C23E1847003EE62F0D89002013C353F
:10091000E926000EEA22EECF06F0EFCF07F00650F0
:100920000E24026E07500F20036E000E1020046E7E
:10093000000E1120056E05C050F204C04FF203C036
:100940004EF202C04DF2000197D0040E355C23E157
:10095000827203EE62F0D89002013D35E926000E66
:10096000EA22EECF06F0EFCF07F006500E24026E1B
:1009700007500F20036E000E1020046E000E112091
:10098000056E05C054F204C053F203C052F202C017
:1009900051F2000171D0050E355C23E1827603EE41
:1009A00062F0D89002013E35E926000EEA22EECF31
:1009B00006F0EFCF07F006500E24026E07500F200E
:1009C000036E000E1020046E000E1120056E05C08F
:1009D00058F204C057F203C056F202C055F20001AB
:1009E0004BD0060E355C23E1837203EE62F0D890A3
:1009F00002013F35E926000EEA22EECF06F0EFCFE6
:100A000007F006500E24026E07500F20036E000EF2
:100A10001020046E000E1120056E05C05CF204C0AB
:100A20005BF203C05AF202C059F2000125D0070E52
:100A3000355C21E1827A03EE62F0D8900201403504
:100A4000E926000EEA22EECF06F0EFCF07F00650BF
:100A50000E24026E07500F20036E000E1020046E4D
:100A6000000E1120056E05C060F204C05FF203C0E5
:100A70005EF202C05DF200010FD80CD011AC0AD0BA
:100A8000116A106A0F6A0E6A02EE41F0200EEE68DB
:100A9000E82EFDD70CEF01F03568348E176A080E8A
:100AA000175C33E2D8901734E96EEA6AEA36E93621
:100AB000EA36410EE926020EEA22EFCF02F0ECCF31
:100AC00003F0ECCF04F0ECCF05F03150025C325073
:100AD0000358335004583450055815E2D890173451
:100AE000E96EEA6AEA36E936EA36410EE926020E8E
:100AF000EA22EFCF31F0ECCF32F0ECCF33F0ECCF95
:100B000034F017C035F0172ACAE3020161910001E1
:100B100012001D681200010E215C02E1D4D818D029
:100B2000020E215C02E173D913D0030E215C01E1B6
:100B30000FD0040E215C01E10BD0050E215C01E118
:100B400007D0060E215C01E103D0070E215C00E115
:100B50002168120023681200226812000D0E1F5C2B
:100B600039E102013A53000133E002014869476963
:100B700046694569376B378320A03793378720A2B2
:100B80003797378B20A4379BC00E801637518012C1
:100B900002EE62F0D8902B34E926000EEA22EECF66
:100BA00006F0EFCF07F006500E24026E07500F201C
:100BB000036E000E1020046E000E1120056E05C09D
:100BC00044F204C043F203C042F202C041F2618128
:100BD000000150D0190E1F5C09E1205080082B6ED7
:100BE000800E2B5C02E37F0E2B6E44D01A0E1F5C2E
:100BF00009E1205080082A6E800E2A5C02E37F0EF5
:100C00002A6E38D0420E1F5C0BE1205203E1259082
:100C100033D804D02580040162818A8200012AD061
:100C2000450E1F5C0CE1205206E1040162918D9497
:100C30008D90000102D00401628100011BD07B0E67
:100C40001F5C17E189928996899A8990899489987D
:100C50008B928D948D908C928B968C968B9A0201B0
:100C60003A6B376B02EE41F0200EEE68E82EFDD7AE
:100C7000618100011F68120002EE41F0200EEE6853
:100C8000E82EFDD789928996899A8D928B908B94C4
:100C90008C908C948B988C988990899489988B925D
:100CA0008D948D908C928B968C968B9A8A924A0E0C
:100CB0002B6E400E2A6E02013A6B376B6181040184
:100CC000628100011200176A360E175C08E2F36AAF
:100CD00001EE37F01750F3CFEBFF172AF5E3070EBD
:100CE00001016B6F060E6C6F050E6D6F040E6E6F5B
:100CF000020E6F6F010E706F716B070E726F060E32
:100D0000736F050E746F040E756F020E766F010E11
:100D1000776F786B050E796F040E7A6F020E7B6F1A
:100D2000010E7C6F7D6B020E7E6F010E7F6F806BFC
:100D3000040E816F020E826F010E836F846B020EB0
:100D4000856F040E866F020E876F010E886F896BA8
:100D5000020E8A6F010E8B6F8C6B040E8D6F020E6C
:100D60008E6F010E8F6F906B020E916F040E926F5B
:100D7000020E936F010E946F956B5F0E176E00015C
:100D8000800E175C08E2F36A01EE37F01750F3CFDC
:100D9000EBFF172AF4E3176A800E175C24E201EEDA
:100DA00037F01750EB500101366F36510001E8A4BF
:100DB00003D00101368B3695010136510001E8A2BE
:100DC00003D001013687369301013631000103E378
:100DD000010136833691000101EE37F0175036C11C
:100DE000EBFF172AD9E3176A800E175C0FE201EEBA
:100DF00037F01750EB50066ED8900630026E01EEB9
:100E0000B7F0175002C0EBFF172AEEE31200176A83
:100E1000340E175C08E2F36A01EE37F01750F3CF97
:100E2000EBFF172AF5E301016A6B070E6B6F060EE5
:100E30006C6F050E6D6F040E6E6F020E6F6F010EFC
:100E4000706F716B070E726F060E736F050E746F05
:100E5000040E756F020E766F010E776F786B050EBC
:100E6000796F040E7A6F020E7B6F010E7C6F7D6BC3
:100E7000020E7E6F010E7F6F806B040E816F020E7B
:100E8000826F010E836F846B020E856F040E866F76
:100E9000020E876F010E886F896B020E8A6F010E3A
:100EA0008B6F8C6B040E8D6F020E8E6F010E8F6F29
:100EB000906B020E916F040E926F020E936F010EF3
:100EC000946F956B5F0E176E0001800E175C08E241
:100ED000F36A01EE37F01750F3CFEBFF172AF4E374
:100EE000010E176E800E175C0EE21704066E01EEFF
:100EF00037F01750EBCF02F001EE37F0065002C08A
:100F0000EBFF172AEFE3176A800E175C24E201EE6D
:100F100037F01750EB500101366F36510001E8A44D
:100F200003D00101368B3695010136510001E8A24C
:100F300003D001013687369301013631000103E306
:100F4000010136833691000101EE37F0175036C1AA
:100F5000EBFF172AD9E3176A800E175C0FE201EE48
:100F600037F01750EB50066ED8900630026E01EE47
:100F7000B7F0175002C0EBFF172AEEE31200020190
:100F8000636962695C0E656F7A0E646F590E676FF4
:100F9000850E666F580E696F140E686F560E6B6F74
:100FA000A90E6A6F550E6D6F430E6C6F530E6F6F07
:100FB000E30E6E6F520E716F890E706F510E736F6C
:100FC000350E726F4F0E756FE60E746F4E0E776FA3
:100FD0009C0E766F4D0E796F580E786F4C0E7B6FAE
:100FE000190E7A6F4A0E7D6FDF0E7C6F490E7F6F90
:100FF000AA0E7E6F480E816F7A0E806F470E836F48
:101000004F0E826F460E856F290E846F450E876FD7
:10101000080E866F430E896FEB0E886F420E8B6F42
:10102000D30E8A6F410E8D6FBF0E8C6F400E8F6F87
:10103000B00E8E6F3F0E916FA50E906F3E0E936FA8
:101040009E0E926F3D0E956F9C0E946F3C0E976FA7
:101050009E0E966F3B0E996FA40E986F3A0E9B6F83
:10106000AE0E9A6F390E9D6FBC0E9C6F380E9F6F3F
:10107000CE0E9E6F370EA16FE30EA06F360EA36FDC
:10108000FD0EA26F360EA56F1A0EA46F350EA76F58
:101090003B0EA66F340EA96F5F0EA86F330EAB6FB9
:1010A000870EAA6F320EAD6FB20EAC6F310EAF6FFE
:1010B000E10EAE6F310EB16F140EB06F300EB36F24
:1010C000490EB26F2F0EB56F820EB46F2E0EB76F32
:1010D000BE0EB66F2D0EB96FFD0EB86F2D0EBB6F25
:1010E0003F0EBA6F2C0EBD6F850EBC6F2B0EBF6FFF
:1010F000CD0EBE6F2B0EC16F180EC06F2A0EC36FC0
:10110000670EC26F290EC56FB80EC46F290EC76F68
:101110000C0EC66F280EC96F620EC86F270ECB6FFC
:10112000BC0ECA6F270ECD6F180ECC6F260ECF6F78
:10113000760ECE6F250ED16FD80ED06F250ED36FE1
:101140003C0ED26F240ED56FA20ED46F240ED76F33
:101150000B0ED66F230ED96F760ED86F220EDB6F73
:10116000E40EDA6F220EDD6F540EDC6F210EDF6F9E
:10117000C60EDE6F210EE16F3B0EE06F200EE36FB7
:10118000B20EE26F200EE56F2B0EE46F1F0EE76FBD
:10119000A60EE66F1F0EE96F240EE86F1E0EEB6FB2
:1011A000A30EEA6F1E0EED6F250EEC6F1D0EEF6F96
:1011B000A90EEE6F1D0EF16F2E0EF06F1C0EF36F69
:1011C000B60EF26F1C0EF56F3F0EF46F1B0EF76F2D
:1011D000CB0EF66F1B0EF96F580EF86F1A0EFB6FE1
:1011E000E80EFA6F1A0EFD6F790EFC6F1A0EFF6F84
:1011F0000B0EFE6F190E0301016FA00E006F190E8A
:10120000036F360E026F180E056FCE0E046F180EA8
:10121000076F680E066F180E096F030E086F170E22
:101220000B6FA00E0A6F170E0D6F3F0E0C6F160E90
:101230000F6FDF0E0E6F160E116F800E106F160EF1
:10124000136F240E126F150E156FC80E146F150E46
:10125000176F6E0E166F150E196F160E186F140E8F
:101260001B6FBF0E1A6F140E1D6F690E1C6F140ECC
:101270001F6F150E1E6F130E216FC20E206F130EFF
:10128000236F710E226F130E256F210E246F120E25
:10129000276FD20E266F120E296F840E286F120E42
:1012A0002B6F380E2A6F110E2D6FED0E2C6F110E55
:1012B0002F6FA30E2E6F110E316F5A0E306F110E5D
:1012C000336F120E326F100E356FCC0E346F100E5E
:1012D000376F870E366F100E396F420E386F0F0E54
:1012E0003B6F3A693D6FBD0E3C6F0F0E3F6F7C0E3A
:1012F0003E6F0F0E416F3D0E406F0E0E436FFE0EA0
:10130000426F0E0E456FC00E446F0E0E476F830E78
:10131000466F0E0E496F470E486F0E0E4B6F0C0E48
:101320004A6F0D0E4D6FD20E4C6F0D0E4F6F990E12
:101330004E6F0D0E516F610E506F0D0E536F2A0ED2
:10134000526F0C0E556FF40E546F0C0E576FBE0E8D
:10135000566F0C0E596F8A0E586F0C0E5B6F560E3F
:101360005A6F0C0E5D6F230E5C6F0B0E5F6FF10EEC
:101370005E6F0B0E616FC00E606F176A0001800E0A
:10138000175C24E202EE62F0D8901734E926000ED2
:10139000EA22EECF06F0EFCF07F00730036E0630FB
:1013A000026E0332023203320232033202320F0E75
:1013B000031602EE62F0D8901734E926000EEA22F6
:1013C00002C0EEFF03C0EFFF172AD8E303016369F1
:1013D0006269A20E656FC30E646F9A0E676F460E48
:1013E000666F960E696F320E686F920E6B6F3A0ED3
:1013F0006A6F8E0E6D6F5D0E6C6F8A0E6F6F9A0E38
:101400006E6F860E716FF00E706F830E736F5F0ECE
:10141000726F7F0E756FE70E746F7C0E776F850E9F
:10142000766F790E796F3B0E786F760E7B6F070EB5
:101430007A6F720E7D6FE80E7C6F6F0E7F6FDF0E1E
:101440007E6F6C0E816FEA0E806F6A0E836F0A0EDC
:10145000826F670E856F3C0E846F640E876F820EFD
:10146000866F610E896FDA0E886F5F0E8B6F440E88
:101470008A6F5C0E8D6FBF0E8C6F5A0E8F6F4C0E85
:101480008E6F570E916FE90E906F550E936F960EFB
:10149000926F530E956F946F510E976F200E966F4B
:1014A0004E0E996FFB0E986F4C0E9B6FE50E9A6F68
:1014B0004A0E9D6FDC0E9C6F480E9F6FE20E9E6F72
:1014C000460EA16FF50EA06F450EA36F150EA26F0D
:1014D000430EA56F420EA46F410EA76F7B0EA66F41
:1014E0003F0EA96FC00EA86F3E0EAB6F100EAA6F15
:1014F0003C0EAD6F6D0EAC6F3A0EAF6FD40EAE6F8B
:10150000390EB16F460EB06F370EB36FC20EB26FA9
:10151000360EB56F490EB46F340EB76FDA0EB66F74
:10152000330EB96F740EB86F320EBB6F180EBA6FF0
:10153000300EBD6FC50EBC6F2F0EBF6F7B0EBE6F22
:101540002E0EC16F3A0EC06F2D0EC36F020EC26F0A
:101550002B0EC56FD10EC46F2A0EC76FA90EC66FB2
:10156000290EC96F880EC86F280ECB6F6F0ECA6F19
:10157000270ECD6F5E0ECC6F260ECF6F530ECE6F43
:10158000250ED16F500ED06F240ED36F540ED26F34
:10159000230ED56F5E0ED46F220ED76F6F0ED66FEF
:1015A000210ED96F860ED86F200EDB6FA30EDA6F77
:1015B0001F0EDD6FC60EDC6F1E0EDF6FEF0EDE6FCF
:1015C0001E0EE16FE06F1D0EE36F520EE26F1C0EF8
:1015D000E56F8C0EE46F1B0EE76FCB0EE66F1B0EF4
:1015E000E96F0F0EE86F1A0EEB6F580EEA6F190EC7
:1015F000ED6FA50EEC6F180EEF6FF80EEE6F180E74
:10160000F16F4F0EF06F170EF36FAB0EF26F170EF8
:10161000F56F0A0EF46F160EF76F6F0EF66F150E5C
:10162000F96FD70EF86F150EFB6F430EFA6F140E9D
:10163000FD6FB30EFC6F140EFF6F270EFE6F130EBF
:101640000401016F9F0E006F130E036F1A0E026FDD
:10165000120E056F990E046F120E076F1B0E066FA8
:10166000110E096FA10E086F110E0B6F290E0A6F74
:10167000100E0D6FB50E0C6F100E0F6F440E0E6F27
:101680000F0E116FD60E106F0F0E136F6B0E126FC1
:101690000F0E156F030E146F0E0E176F9D0E166F43
:1016A0000E0E196F3A0E186F0D0E1B6FDA0E1A6FB1
:1016B0000D0E1D6F7C0E1C6F0D0E1F6F210E1E6F09
:1016C0000C0E216FC80E206F0C0E236F720E226F4E
:1016D0000C0E256F1E0E246F0B0E276FCC0E266F7F
:1016E0000B0E296F7C0E286F0B0E2B6F2E0E2A6FA0
:1016F0000A0E2D6FE30E2C6F0A0E2F6F990E2E6FB0
:101700000A0E316F510E306F0A0E336F0B0E326FAF
:10171000090E356FC80E346F090E376F850E366FA0
:10172000090E396F450E386F090E3B6F060E3A6F82
:10173000080E3D6FC90E3C6F080E3F6F8E0E3E6F58
:10174000080E416F540E406F080E436F1C0E426F1F
:10175000070E456FE50E446F070E476FAF0E466FDD
:10176000070E496F7B0E486F070E4B6F490E4A6F8D
:10177000070E4D6F170E4C6F060E4F6FE70E4E6F34
:10178000060E516FB90E506F060E536F8B0E526FCF
:10179000060E556F5F0E546F060E576F340E566F60
:1017A000060E596F0A0E586F050E5B6FE10E5A6FE9
:1017B000050E5D6FB90E5C6F050E5F6F930E5E6F69
:0E17C000050E616F6D0E606F00011200FFD705
:020000040030CA
:0300010006160ED2
:020005008580F4
:060008000FC00FE00F40E5
:00000001FF
